:04000000A7EF07F06F
:1000080000C015F0E1CF16F0E2CF17F09EAA4AD053
:100018009DAA48D0AECF1CF0ABA202D0AB98AB885B
:10002800ABA403D0AECF1CF01C6A1C500D0A13E120
:10003800010E186E000E196E780E1A24E16E000E6D
:100048001B20E26EE66A1AC01DF01BC01EF01A6A79
:100058001B6A1C6A0ED0780E1A24E16E000E1B2053
:10006800E26E1CC0E6FF1AC01DF01BC01EF01A4A43
:100078001B2A000E1B5C02E1800E1A5C13E3020EC1
:10008800186E000E196E9D9A780E1A24E16E000EF5
:100098001B20E26EE66A1AC01DF01BC01EF01A6A29
:1000A8001B6A1C6A15C000F016C0E1FF17C0E2FF0A
:0200B800110035
:0C00BA0072B201D0FDD7C0C173FF12006C
:0E00C600ACB202D00000FCD7C0C1ADFF1200EA
:1000D400F250026EF29E0500FF6A0150FE6E00505F
:0800E400FD6E02BEF28E120057
:1000EC00C7B409D01F0EC514016E0150000A03E1FC
:0A00FC00010E006E01D0006A120030
:04010600C58412009A
:10010A009E96BAC1C9FF1FC0BBF120C0BCF121C075
:10011A00BDF122C0BEF1C7A421D01F50201021106A
:10012A0022101BE00101BB51BC11BD11BE110EE131
:10013A008BC1E1FF8CC1E2FF040EE66E89C100F0BB
:10014A008AC101F0C2DF010E006E3AD0010E010130
:10015A00BB5F000EBC5BBD5BBE5BDDD71FC0BBF1E6
:10016A0020C0BCF121C0BDF122C0BEF19EB621D093
:10017A001F502010211022101BE00101BB51BC119D
:10018A00BD11BE110EE18BC1E1FF8CC1E2FF040E6D
:10019A00E66E89C100F08AC101F097DF010E006E98
:1001AA000FD0010E0101BB5F000EBC5BBD5BBE5BE5
:1001BA00DDD7C5BC02D0006A03D0C584020E006E2A
:0201CA00120021
:1001CC001FC0BCF120C0BDF121C0BEF122C0BFF1E7
:1001DC000101BA6BBB6BBB51120802E1BA518E081C
:1001EC0008E37EDF005201E004D00101BA4BBB2BC7
:1001FC00F2D70101120EBB5D02E18F0EBA5D03E373
:10020C007B0E006E24D0C580C5A020D01F502010BE
:10021C00211022101AE0BC51BD11BE11BF110EE10C
:10022C008BC1E1FF8CC1E2FF050EE66E89C100F0C7
:10023C008AC101F049DF010E006E09D0010E0101E7
:10024C00BC5F000EBD5BBE5BBF5BDED7006A1200FD
:10025C00B7DFB7C1BAF153DF00C0B9F1000E016EC0
:10026C00FF0E011802E1FF0E0018D8B4C69EB8C1EB
:10027C00BAF145DF00C0B9F140DFB9C100F012009E
:10028C00F00E0101B515006E0086008000C0B6F1BD
:10029C0077C0B7F1040E0010B86FDADF00C09BF125
:1002AC00000E01019C6F060E0D6E0D2EFED7000088
:1002BC0077C0B7F1FB0EB615B86FCADF00C09BF163
:1002CC00000E01019C6F060E0D6E0D2EFED7000068
:1002DC00B5C100F00036009000360090003600905A
:1002EC0000360090F00E00160086008000C0B6F1BB
:1002FC0077C0B7F1040E0010B86FAADF00C09BF1F5
:10030C00000E01019C6F060E0D6E0D2EFED7000027
:10031C0077C0B7F1FB0EB615B86F9ADF00C09BF132
:10032C00000E01019C6F100E0D6E0D2EFED70000FD
:02033C001200AD
:10033E00086A080E0C6E003408360450085ED8B0F9
:0E034E0002D00826D89000360C2EF5D71200EB
:10035C00AFC1F6FFB0C1F7FFB1C1F8FF0900F5CF8F
:10036C0000F0005210E0AFC1F6FFB0C1F7FFB1C111
:10037C00F8FF0900F5CFB5F183DF010EAF27000EB2
:08038C00B023B123E5D71200F4
:10039400F00E0101AF15006E008600C0B1F177C008
:1003A400B7F1040E0010B86F57DF00C09BF1000EC8
:1003B40001019C6F210E0D6E0D2EFED777C0B7F193
:1003C400FB0EB115B86F48DF00C09BF1000E0101B0
:1003D4009C6F210E0D6E0D2EFED7B051010A34E133
:1003E400AFC100F000360090003600900036009057
:1003F40000360090F00E0016008600C0B1F177C000
:10040400B7F1040E0010B86F27DF00C09BF1000E97
:1004140001019C6F060E0D6E0D2EFED7000077C0F5
:10042400B7F1FB0EB115B86F17DF00C09BF1000EDA
:1004340001019C6F0D0E0C6EFB0E0D6E0D2EFED782
:0A0444000C2EFCD70000000012008F
:10044E000101B26B030EB25D0AE2B251B025E16E4C
:10045E00000EB121E26E200EE66EB22BF3D7B25132
:10046E00B025E16E000EB121E26EE66AB207B2511E
:10047E00B025B36F000EB121B46F0A0E046EAFC17A
:10048E0000F056DF08C000F0300E0026B3C1E1FFC9
:10049E00B4C1E2FF00C0E6FF0A0E046EAFC100F069
:1004AE0047DF00C0AFF10050000A01E102D0B207F1
:0404BE00DED7120073
:1004C200086A096A100E0C6E0134083609360450A7
:1004D200085E0550D8A0053C095ED8B007D004508C
:1004E20008260550D8B0053C0926D89000360136BA
:0604F2000C2EEAD71200F7
:1004F8000D0E0101C06FE3DD0A0E0101C06FDFDDE3
:020508001200DF
:10050A00AFC1F6FFB0C1F7FFB1C1F8FF0900F5CFDF
:10051A0000F0005211E0AFC1F6FFB0C1F7FFB1C160
:10052A00F8FF0900F5CFC0F1C9DD010E0101AF27BF
:0A053A00000EB023B123E4D7120035
:100544000B6A0A6A096A086A0E6A03340836045098
:10055400085E0550D8A0053C095E0650D8A0063CAC
:100564000A5E0750D8A0073C0B5EE86AD8A0010ECB
:100574000E5E0336070E0C6E0334083609360A364F
:100584000B360E36045003A012D0085E0550D8A0D6
:10059400053C095E0650D8A0063C0A5E0750D8A068
:1005A400073C0B5EE86AD8A0010E0E5E11D0082647
:1005B4000550D8B0053C09260650D8B0063C0A269A
:1005C4000750D8B0073C0B26E86AD8B0010E0E26B7
:1005D40003360C2ED1D70234083609360A360B36C8
:1005E4000E36045003A012D0085E0550D8A0053C76
:1005F400095E0650D8A0063C0A5E0750D8A0073C06
:100604000B5EE86AD8A0010E0E5E11D008260550D4
:10061400D8B0053C09260650D8B0063C0A26075037
:10062400D8B0073C0B26E86AD8B0010E0E26023675
:10063400070E0C6E0234083609360A360B360E36AF
:10064400045002A012D0085E0550D8A0053C095EF3
:100654000650D8A0063C0A5E0750D8A0073C0B5EA3
:10066400E86AD8A0010E0E5E11D008260550D8B055
:10067400053C09260650D8B0063C0A260750D8B0D7
:10068400073C0B26E86AD8B0010E0E2602360C2E63
:10069400D1D70134083609360A360B360E360450E3
:1006A40002A012D0085E0550D8A0053C095E065091
:1006B400D8A0063C0A5E0750D8A0073C0B5EE86A47
:1006C400D8A0010E0E5E11D008260550D8B0053C06
:1006D40009260650D8B0063C0A260750D8B0073C75
:1006E4000B26E86AD8B0010E0E260136070E0C6EF2
:1006F4000134083609360A360B360E36045001A08A
:1007040012D0085E0550D8A0053C095E0650D8A05A
:10071400063C0A5E0750D8A0073C0B5EE86AD8A0E6
:10072400010E0E5E11D008260550D8B0053C0926EE
:100734000650D8B0063C0A260750D8B0073C0B2612
:10074400E86AD8B0010E0E2601360C2ED1D700343B
:10075400083609360A360B360E36045001A012D07C
:10076400085E0550D8A0053C095E0650D8A0063C9A
:100774000A5E0750D8A0073C0B5EE86AD8A0010EB9
:100784000E5E11D008260550D8B0053C0926065047
:10079400D8B0063C0A260750D8B0073C0B26E86AB6
:1007A400D8B0010E0E260036070E0C6E0034083643
:1007B40009360A360B360E36045000A012D0085EF5
:1007C4000550D8A0053C095E0650D8A0063C0A5E38
:1007D4000750D8A0073C0B5EE86AD8A0010E0E5E55
:1007E40011D008260550D8B0053C09260650D8B0CB
:1007F400063C0A260750D8B0073C0B26E86AD8B056
:10080400010E0E2600360C2ED1D700B00ED00450A7
:1008140008260550D8B0053C09260650D8B0063C39
:0C0824000A260750D8B0073C0B26120033
:100830000101B26BAFC1E9FFB0C1EAFFEECFB1F188
:10084000B151000A0EE0B1C1C0F13DDC0101B22B93
:10085000B251AF25E96E000EB021EA6EEECFB1F1D4
:04086000EFD71200BC
:10086400C60E0101916F000E926FC00E936F010EC0
:10087400946FFF0E9D6FFF0E9E6F000E9F6F000E14
:10088400A06FFF0EA16FFF0EA26F000EA36F000EEC
:10089400A46F9A0E976F090E986F000E996F000E51
:1008A4009A6FAC8A900EAB6E948E949C9EAA03D0E1
:0808B400AECF00F0FBD71200EB
:1008BC000101AB6BAC6B000EAC5D02E10A0EAB5DE3
:1008CC000BE2AB51A925E16EAC51AA21E26E200ED0
:1008DC00E66EAB4BAC2BEFD7AB51A925E16EAC510F
:1008EC00AA21E26EE66A010EAB5F000EAC5BAB5167
:1008FC00A925AD6FAC51AA21AE6F0A0E046E000E85
:10090C00056E066E076EA5C100F0A6C101F0A7C169
:10091C0002F0A8C103F010DE08C000F009C001F01D
:10092C000AC002F00BC003F0300E0026ADC1E1FF8F
:10093C00AEC1E2FF00C0E6FF0A0E046E000E056EAB
:10094C00066E076EA5C100F0A6C101F0A7C102F0AA
:10095C00A8C103F0F1DD00C0A5F101C0A6F102C0F1
:10096C00A7F103C0A8F1000E046E031808E10450AF
:10097C00021805E10450011802E10050000A01E1DF
:0E098C0005D0010EAB5F000EAC5BB1D71200C0
:0A099A00000EACB2010E006E120058
:1009A400EC0E01018D6F000E8E6F000E8F6F000E26
:1009B400906FCC0E2B6E010E2C6E000E2D6E000E61
:1009C4002E6EFF0E00016F6FFF0E706F000E716FC1
:1009D400000E726FFF0E236EFF0E246EFF0E256E47
:1009E400FF0E266E0A0E276E010E286EBA0E296EB1
:1009F400010E2A6E060E736F010E746F000E756F72
:100A0400000E766F949894968B988B96948894861F
:0A0A1400C79EC79C380EC66E120084
:100A1E00030E806E0F01386B38813883030E926E91
:100A2E00806A826A3A6BFF0E946E948E949C3C6B35
:100A3E00966AFF0E846E836A956A3B6B9C981200D1
:100A4E000900F5CFE6FF0006FBE10106F9E1120011
:100A5E000101A66B890EAF6F160EB06F000EB16F4F
:100A6E004DDDA5C1AFF12F0E0101B06F000EB16FBC
:100A7E00E7DC2F0EAF6F000EB06FD3DEE6EC00F0AA
:100A8E00A5C1BAF185EC00F00050000A09E0450E50
:100A9E000101AF6F170EB06F000EB16F2FDD0BD0CF
:100AAE005E0E0101AF6F170EB06F000EB16F26DD37
:100ABE00010E0101A66F83EC00F017DDA6C100F058
:020ACE00120014
:100AD000A5C104F0A6C105F00101A951AA1124E0A5
:100AE000010EA95F000EAA5B04C002F005C003F06E
:100AF000044A052AA7C100F0A8C101F0A74BA82B02
:100B000000C0E9FF01C0EAFF02C0E1FF03C0E2FF4D
:100B1000EECFE6FF02C0E9FF03C0EAFFEECF00F030
:100B2000005201E101D0D8D7A9C100F0AAC101F05B
:100B3000010EA95F000EAA5B0050011008E004C07E
:100B4000E1FF05C0E2FFE66A044A052AEDD7A5C128
:080B500000F0A6C101F0120043
:100B5800A5C102F0A6C103F002C000F003C001F075
:100B6800024A032A00C0E9FF01C0EAFFEE5201E091
:100B7800F3D70101A551025C006EA6510358016E1E
:0A0B8800010E005E000E015A12007B
:100B92000101A96B050EA95D0AE2A951A725E16E23
:100BA200000EA821E26E200EE66EA92BF3D7A95102
:100BB200A725E16E000EA821E26EE66AA907A951F7
:100BC200A725AA6F000EA821AB6F0A0E046E000EB5
:100BD200056EA5C100F0A6C101F072DC08C000F0EC
:100BE20009C001F0300E0026AAC1E1FFABC1E2FF4D
:100BF20000C0E6FF0A0E046E000E056EA5C100F0ED
:100C0200A6C101F05DDC00C0A5F101C0A6F1000E95
:100C1200011802E1000E001801E102D0A907CFD7A6
:020C22001200BE
:100C24000101A76BA86BA751A525E96EA851A621C0
:100C3400EA6EEE50000A16E0800EA819006E800ECF
:100C4400005C02E1140EA75D0DE2A751A525E96E33
:100C5400A851A621EA6EEECFB5F146EC01F0A74B00
:060C6400A82BE1D71200ED
:100C6A00A5C195F1A6C196F1A7C101F0010E006ECA
:100C7A00015004E000360090FF0FFBD700C000F1DE
:100C8A00001E00C0FFF0120E0101A525E96E000E3C
:100C9A00A621EA6E0050EF16120EE95E0050EF161A
:020CAA00120036
:100CAC00A7C1F6FFA8C1F7FFA9C1F8FF0900F5CF4E
:100CBC0000F0005218E0A7C1F6FFA8C1F7FFA9C1C8
:100CCC00F8FF0900F5CF00F0A5C1E1FFA6C1E2FFD6
:100CDC0000C0E6FF0101A54BA62B010EA727000EB5
:100CEC00A823A923DDD7A5C1E1FFA6C1E2FFE66ACF
:020CFC001200E4
:100CFE00300E0101C06F63EC00F0020E0B6E040E9D
:100D0E000C6EBA0E0D6E0D2EFED70C2EFCD70B2EC2
:100D1E00FAD70000300E0101AF6FB06BCAEC01F0D4
:100D2E00310EC06F63EC00F0410E0C6EEE0E0D6EC8
:100D3E000D2EFED70C2EFCD70000300E0101AF6F2A
:100D4E00B06BCAEC01F0320EC06F63EC00F0410ED6
:100D5E000C6EEE0E0D6E0D2EFED70C2EFCD7000077
:100D6E00300E0101AF6FB06BCAEC01F0330EC06FE5
:100D7E0063EC00F0410E0C6EEE0E0D6E0D2EFED7D6
:100D8E000C2EFCD70000250E0101AF6FB06BCAEC24
:100D9E0001F0340EC06F63EC00F0340E0C6EF10EE9
:100DAE000D6E0D2EFED70C2EFCD700000000280E67
:100DBE000101AF6F010EB06FCAEC01F0350EC06FBE
:100DCE0063EC00F0340E0C6EF10E0D6E0D2EFED790
:100DDE000C2EFCD700000000080E0101AF6F010EB3
:100DEE00B06FCAEC01F0360EC06F63EC00F0340E3B
:100DFE000C6EF10E0D6E0D2EFED70C2EFCD70000D4
:100E0E000000010E0101AF6F010EB06FCAEC01F0D0
:100E1E00370EC06F63EC00F0020E0B6E040E0C6EFC
:100E2E00BA0E0D6E0D2EFED70C2EFCD70B2EFAD74A
:100E3E000000060E0101AF6F010EB06FCAEC01F09B
:100E4E00380EC06F63EC00F0340E0C6EF10E0D6EAA
:100E5E000D2EFED70C2EFCD7000000000C0E01014B
:100E6E00AF6F010EB06FCAEC01F0390EC06F63ECBC
:100E7E0000F0340E0C6EF10E0D6E0D2EFED70C2EF4
:0C0E8E00FCD7000000007CEC02F0120019
:100E9A009D9A1A6A1B6A000E1B5C02E1800E1A5C9C
:100EAA000AE2780E1A24E16E000E1B20E26EE66A50
:100EBA001A4A1B2AF0D71A6A1B6A1D6A1E6AAECF23
:0C0ECA001CF01C6A186A196A9D8A12004C
:100ED6002DD0800E0101AF6F010EB06FCAEC01F08C
:100EE600B30EAF6F160EB06F000EB16FAEEC01F021
:100EF600800E0101AF6F010EB06FCAEC01F023D076
:100F0600C00EAF6F010EB06FCAEC01F0740EAF6F7A
:100F1600160EB06F000EB16FAEEC01F0C00E0101FF
:100F2600AF6F010EB06FCAEC01F00DD00101000EDB
:100F3600A61902E1010EA519CCE0000EA61902E1E0
:080F4600020EA519DDE0120006
:100F4E00C2EC0BF0D38CD38AD398D382D390D3B484
:100F5E0001D0FDD75DDD8998070E0101876F010E67
:100F6E00886FB886B06A670EAF6EAC8474DC020E02
:100F7E000B6E040E0C6EBA0E0D6E0D2EFED70C2ED1
:100F8E00FCD70B2EFAD7000001DD0050010A06E156
:100F9E0001010D0EC06F63EC00F0F6D70C0E0101CF
:100FAE00C06F63EC00F00B0E0B6E260E0C6E5D0E1A
:100FBE000D6E0D2EFED70C2EFCD70B2EFAD7000081
:100FCE0000007CEC02F05A0E0101AF6F160EB06FEE
:100FDE00000EB16F85EC02F0DC0E0101AF6F160E44
:100FEE00B06F000EB16F85EC02F0710E0101AF6FA4
:100FFE00150EB06F000EB16F85EC02F0400E0101C0
:10100E00AF6F160EB06F000EB16F85EC02F0260EAC
:10101E000101AF6F160EB06F000EB16F85EC02F0CE
:10102E003B0E0101AF6F150EB06F000EB16F85EC68
:10103E0002F0040E0101AF6F150EB06F000EB16F0E
:10104E0085EC02F0400E0001FB6F1F0EFC6F000ED0
:10105E00FD6FFE6F700E0101AF6F170EB06F000EB9
:10106E00B16F85EC02F0FBC0A5F1FCC0A6F1FDC08E
:10107E00A7F1FEC0A8F187C1A9F188C1AAF117DCBA
:10108E0087C1AFF188C1B0F118EC04F0780EAF6FE4
:10109E00170EB06F000EB16F85EC02F0A50E0101B8
:1010AE00AF6F150EB06F000EB16F85EC02F0230E10
:1010BE000101C06F63EC00F07CEC02F0330E0B6E9E
:1010CE00BB0E0C6EDF0E0D6E0D2EFED70C2EFCD74A
:1010DE000B2EFAD700000000400E0101C06F63EC2A
:1010EE0000F07CEC02F0C80E0101AF6F160EB06F6F
:1010FE00000EB16F85EC02F0140EC86E4CDC060EBD
:10110E000B6E130E0C6EAD0E0D6E0D2EFED70C2E3D
:10111E00FCD70B2EFAD700000000300EF96F000E30
:10112E00FA6F000EFA5D02E1800EF95D17E2F9C06A
:10113E00A5F18EDC0050010A01E110D0820E0C6E7A
:10114E00DD0E0D6E0D2EFED70C2EFCD7000000000E
:10115E00020E0001F927000EFA23E3D7020E0B6EE2
:10116E00040E0C6EBA0E0D6E00010D2EFDD70C2E58
:10117E00FBD70B2EF9D700004A0EF86F4A0E776F89
:10118E000C0E0101AF6F160EB06F000EB16F85EC35
:10119E0002F0AEDD7CEC02F0010E0101B56F46EC03
:1011AE0001F0040E0B6E0C0E0C6E330E0D6E0D2E2A
:1011BE00FED70C2EFCD70B2EFAD700000000CB0E5C
:1011CE00AF6F150EB06F000EB16F85EC02F087C1D8
:1011DE00A5F188C1A6F1340E0101A76F170EA86FF5
:1011EE00000EA96F5CDD87C1AFF188C1B0F118ECBC
:1011FE0004F07CEC02F0010E0101A56F000EA66F4B
:10120E0063DE010EAF6F170EB06F000EB16FAEEC56
:10121E0001F0EC0E0101AF6F150EB06F000EB16F45
:10122E0085EC02F087C1A5F188C1A6F19E0E0101E1
:10123E00A76F160EA86F000EA96F31DD87C1AFF133
:10124E0088C1B0F118EC04F07CEC02F0020E010142
:10125E00A56F000EA66F38DE120EAF6F170EB06FB1
:10126E00000EB16FAEEC01F0330E0B6EBB0E0C6EBA
:10127E00DF0E0D6E0D2EFED70C2EFCD70B2EFAD7D1
:10128E0000000000010E0101AF6F010EB06FCAEC3D
:10129E0001F0040E0B6E0C0E0C6E330E0D6E0D2E39
:1012AE00FED70C2EFCD70B2EFAD700000000010E35
:1012BE00A56F000EA66F08DEEF0EAF6F160EB06FA5
:1012CE00000EB16FAEEC01F0AB8EAB86AB96D08E4E
:1012DE00F28CF28EDBDD800E0101A56F0F0EA66F74
:1012EE00030EA76FBBDC056B066B000E191802E12F
:1012FE00010E1818D8A4C4D0780EAF6F000EB06FC0
:10130E0018EC04F07CEC02F00001986B780E0101F1
:10131E00A56F000EA66F19DC00C003F101C004F129
:10132E00010EA56F000EA66FCFDD0001F96BFA6BF3
:10133E00010104510001FA5D04E1010103510001B4
:10134E00F95D6FE20F0EF915006EFAC001F0000E96
:10135E0001162F0E0024E16E000E0120E26E780EB3
:10136E00F925E96E000EFA21EA6EEECFE6FFF9C01E
:10137E0001F1FAC002F1010102330133029F02337F
:10138E000133029F02330133029F02330133029F66
:10139E000F0E0001F915016EFAC002F0000E0216D2
:1013AE00000E021802E1000E011837E101C100F033
:1013BE0002C101F0000E026E036E0036009001367F
:1013CE0002360336680E0024F66E170E0120F76EF5
:1013DE00000E0220F86E0900F5CFAFF1010E0101EB
:1013EE00B06FCAEC01F02F0EA56F000EA66F780E2F
:1013FE000001F9250101A76F000E0001FA2101017C
:10140E00A86F100EA96F000EAA6F68EC05F02F0ED4
:10141E00A56F000EA66F12EC06F00001F94BFA2B29
:10142E0087D73D0E0B6EE10E0C6E3F0E0D6E0D2E20
:10143E00FED70C2EFCD70B2EFAD700000000010EA3
:10144E000101AF6F010EB06FCAEC01F0230EAF6F4A
:10145E00170EB06F000EB16FAEEC01F02F6A186A66
:10146E00196A780E1A24E16E000E1B20E26EE66AEF
:10147E001AC01DF01BC01EF01A6A1B6A1C6A9D8AD8
:10148E000B0E0B6E260E0C6E5D0E0D6E0D2EFED718
:10149E000C2EFCD70B2EFAD7000000007F0E010198
:1014AE00AF6F170EB06F000EB16F85EC02F005C175
:1014BE00A5F106C1A6F12F0E0101A76F000EA86FB0
:1014CE00C9EC05F02F0EAF6F000EB06F18EC04F0E4
:1014DE007CEC02F08B0E0101AF6F010EB06FCAEC07
:1014EE0001F02F0EA56F000EA66F12EC06F0054B45
:0614FE00062BFBD6FFD710
:1017840010EE18F00B0E006E010E016E530EF66E85
:0E179400170EF76E000EF86E27EC05F012002F
:101504002054657374204C434420313630322032E9
:1015140078313620656E2049324320766961205047
:10152400434638373534206164646974696F6E6E7C
:07153400656C0D0A0D0A00B1
:10153B002055415254312076696120555342202D5C
:10154B003E20434F4D342031393230302C382C4E25
:10155B002C31205465725465726D205465726D691F
:06156B006E616C0D0A0028
:1015710020536F75726365203A5F31384634366B9C
:1015810032325F4C43445F313630325F327831362C
:101591005F493243315F48575F3139303532312E3F
:0415A100630D0A00CC
:1015A50020436865636B2064656C61792064652000
:1015B500353030306D5320656E747265202320659B
:0615C5007420400D0A0035
:1015CB002045637269742E207375722031657265C4
:1015DB00206C69676E65206475204C4344203A206B
:0115EB0000FF
:1015EC002045637269742E207375722032656D20EC
:1015FC006C69676E65206475204C4344203A20006A
:10160C0020496E697420446973706C6179204C4375
:0A161C00442032783136203A2000D5
:10162600204C43442032783136207375722062751F
:0A163600732049324331200D0A00F1
:10164000205049432031384634364B3232204D4306
:0A165000552044697034300D0A0083
:10165A0020496E6974205541525431203139323053
:0A166A00302C382C4E2C310D0A00F4
:101674002020202020202020202020202020202066
:051684002020202000E1
:10168900446576696365206174206164726573736A
:0516990065203A20006D
:10169E007061756C666A756A6F203031323334351D
:0516AE00363738390059
:1016B3002020202020202020202020202020202027
:0516C3002020202000A2
:1016C80020496E69742049324331203130304B68EB
:0416D8007A0D0A007D
:1016DC00204D696B726F632050726F20372E323041
:0316EC000D0A00E4
:1016EF00436F6D7074657572204A3D202020202055
:0216FF002000C9
:1017010048656C6C6F204920616D20616C6976655C
:0117110000D7
:101712007061756C666A756A6F2E667265652E6693
:0117220000C6
:10172300436F6D7074657572204A3D202020202020
:0117330000B5
:1017340048656C6C6F204920616D20616C69766529
:0117440000A4
:0E174500206973206E6F7420666F756E6400ED
:02175300000094
:02175500000092
:011757000091
:0217580000008F
:04175A00000000008B
:0A175E0020666F756E64204F4B008B
:081768008000C0009400D400D1
:0817700020466F7363203D0069
:07177800204B487A0D0A0026
:04177F004A3D2000BF
:020000040030CA
:0D00010028193CFFBF81FF0FC00FE00F402A
:0200000400F00A
:10000000626F6F746C6F61646572626F6F746C6F36
:1000100061646572204D696B726F43FFFFFFFFFFE4
:10002000FFFFFFFFFFFFFFFFFFFFFFFFFFFFFFFFE0
:10003000FFFFFFFFFFFFFFFFFFFFFFFFFFFFFFFFD0
:10004000FFFFFFFFFFFFFFFFFFFFFFFFFFFFFFFFC0
:10005000FFFFFFFFFFFFFFFFFFFFFFFFFFFFFFFFB0
:10006000FFFFFFFFFFFFFFFFFFFFFFFFFFFFFFFFA0
:10007000FFFFFFFFFFFFFFFFFFFFFFFFFFFFFFFF90
:10008000FFFFFFFFFFFFFFFFFFFFFFFFFFFFFFFF80
:10009000FFFFFFFFFFFFFFFFFFFFFFFFFFFFFFFF70
:1000A000FFFFFFFFFFFFFFFFFFFFFFFFFFFFFFFF60
:1000B000FFFFFFFFFFFFFFFFFFFFFFFFFFFFFFFF50
:1000C000FFFFFFFFFFFFFFFFFFFFFFFFFFFFFFFF40
:1000D000FFFFFFFFFFFFFFFFFFFFFFFFFFFFFFFF30
:1000E000FFFFFFFFFFFFFFFFFFFFFFFFFFFFFFFF20
:1000F0007061756C666A756A6F2020202020200070
:00000001FF
